:1000000020C0BDC039C038C037C0ECC05BC172C1B0
:1000100033C0C6C031C030C02FC02EC02DC02CC0D0
:100020002BC090C4A5C4B7C4C1C4CBC4FDC431C5E2
:1000300038C543C553C558C55FC569C56EC575C5C7
:1000400082C511241FBECFE5D1E0DEBFCDBF10E0D9
:10005000A0E6B0E0E8E0FDE002C005900D92AE3908
:10006000B107D9F710E0AEE9B0E001C01D92A43BA2
:10007000B107E1F757D146C6C3CF95B79C7F892B0F
:1000800085BF089582E080BF83BF12BE89E686BF28
:1000900089B7826089BF08951ABA17BA1BBA8FEF61
:1000A00088BB8BB38F608BBB8AB38F608ABBD59ABA
:1000B000D69AD798DF9A87B3836087BB08951FBC11
:1000C00089E18EBD12BC8FEF91E095BD84BD84E1C6
:1000D00090E09BBD8ABD99BD88BD1DBC1CBC80E263
:1000E0008CB90895FC01148282E08187808B108690
:1000F00017868091AB00807F8093AB008FEF809359
:10010000AA008093A6000895FC01148282E08187F2
:10011000808B1086178682E18093AC008093A900C3
:100120000895FC0182818230F9F028F4882341F09F
:10013000813011F50FC08330E1F08430E9F417C04D
:100140008081882321F081E08583168208951582BD
:10015000168208958081882321F0158281E08683AC
:1001600008951582168208951582168208951482C4
:10017000138281E085838683089500000895789432
:100180001F920F920FB60F9211248F9312BE81E02F
:1001900080939F008F910F900FBE0F901F90189526
:1001A00078941F920F920FB60F9211248F939F9302
:1001B0008091B0008C3048F09091AE00933019F4EB
:1001C00091E09093B3001092AE008F5F8093B000E7
:1001D00081E080939E009F918F910F900FBE0F90B2
:1001E0001F9018951F920F920FB60F9211242F9304
:1001F0008F939F938EB5887F8EBD8BB39BB32091D9
:10020000AB002F70907F922B9BBB8F7069F0809119
:10021000A7009091A8009BBD8ABD8091A4009091F9
:10022000A50099BD88BD0EC08091A7009091A8003F
:1002300044969BBD8ABD8091A4009091A5004496F0
:1002400099BD88BD9091AA008091A60098130FC017
:100250008091AA009091A6008923809360008091EC
:10026000A4009091A500019699BD88BD03C08FEFB1
:100270008093600081E090E09DBD8CBD8EB5816073
:100280008EBD8091A000811102C0DD9ADE9A90910E
:10029000A0008091AC00981301C0DD989091A0005F
:1002A0008091A900981301C0DE988091A0008F5F13
:1002B0008093A0009F918F912F910F900FBE0F9070
:1002C0001F9018951F920F920FB60F9211242F9323
:1002D0008F939F938BB32091AA009091600082230B
:1002E00089238BBB9F918F912F910F900FBE0F9001
:1002F0001F9018951F920F920FB60F9211242F93F3
:100300008F939F938BB32091A600909160008223DE
:1003100089238BBB9F918F912F910F900FBE0F90D0
:100320001F901895CF93DF93CDB7DEB7EA970FB63E
:10033000F894DEBF0FBECDBFFE01BB9680E1DF01AA
:100340001D928A95E9F7A8DECF9BFECF83E080B9A6
:100350008FEF8093A6008093AA00E199FECF81E001
:1003600090E0BAD4982EE199FECF80E090E0B4D42A
:10037000682F6370CE010196C6D1B1E09B1206C012
:100380006E816370CE014696BED106C06E816F5FEE
:100390006370CE014696B7D182E06FDE8BB7806482
:1003A0008BBF8DDE619A629A82E18093A90080936F
:1003B000AC0068DE1092B30078940F2EF3EBEF2EB2
:1003C000F0E0FF2EF02D0F2EF1EBCF2EF0E0DF2E20
:1003D000F02D0F2EF0E12F2EF7E23F2EF02D0F2EF5
:1003E000F2E17F2EF02D88248A9408EE1DEF2091F3
:1003F000A1003091A2002115310529F488B38C7F2A
:10040000816088BB06C0215031093093A20020933F
:10041000A100F7018081882309F4BEC01082D601B3
:100420008D919C9184D1882309F4B6C088B38C7FC8
:10043000826088BB3092A2002092A100F6018081E8
:1004400091813DD4682EA82EB12CD6018D919C911E
:10045000F501EE0FFF1F21E030E02C0F3D1FE20FF2
:10046000F31F93A782A78E81861166C02B813C81E2
:100470003A832983C501880F991FBE016F5F7F4FA3
:10048000ABE2B0E0AC0FBD1F8A0F9B1F04D48A857E
:10049000823040F488858150442443948E3F18F084
:1004A000412C01C0412C8989823040F48F858150D4
:1004B000552453948E3F18F0512C01C0512CCE017D
:1004C00008962FDECE010F962CDE8C89811102C09A
:1004D00080EF01C084EF9D89911188609D85911105
:1004E00081609E85911182607FB7442031F04885FC
:1004F00050E0440F551F6CEF03C040E350E0682DFF
:10050000552031F02F8530E0220F331F93EF03C0C9
:1005100020E330E0982DF8945093A8004093A70072
:100520003093A5002093A4006093AA009093A600A6
:100530008093AB0078947FBF8B8D86112DC0888D02
:10054000998D9F8B8E8BC501880F991FBE016A5EA6
:100550007F4FEBE2F0E0EC0FFD1F8E0F9F1F9BD350
:100560002F8D223048F49E8D892F213009F48195FA
:100570008E5E8093AC0002C07092AC002EA122303F
:1005800048F49DA1892F213009F481958E5E8093D6
:10059000A90002C07092A90080919F00882319F0E1
:1005A00010929F00E3D080919E00882301F1109269
:1005B0009E002B853C852F5F3F4F3C872B872A89E8
:1005C0003B892F5F3F4F3B8B2A8B29813A81211535
:1005D000310521F0215031093A8329832E893F8941
:1005E0002115310521F0215031093F8B2E8B2981B6
:1005F0003A81232B31F48D81882319F0CE010196A5
:1006000071DD2E893F89232B31F48A8D882319F0DF
:10061000CE01469679DD8A85843079F42B853C8538
:10062000203D374050F082E08A8719868091AB00E8
:100630008C7F8093AB008092AA008989843079F402
:100640002A893B89203D374050F082E0898B188A07
:100650008091AB00837F8093AB008092A600CF99FE
:10066000C6CEF89480E007C0980121503109E9F71F
:10067000853608F48F5FCF9BF7CF8436F0F0E19991
:10068000FECF91100BC061E081E090E02DD36E8130
:10069000CE01469638D0992493940BC060E081E057
:1006A00090E022D36E816F5F6370CE0146962BD0AF
:1006B000912CCE01469628DD24C08E818F5F0F2EAF
:1006C000F3E0BF2EF02DB8226B2DCE0101961BD08A
:1006D000911007C06B2D6F5F6370CE01469613D0EB
:1006E00004C06B2DCE0146960ED0E199FECF6B2D46
:1006F00080E090E0F9D2CE010196F4DCCE0146967E
:1007000003DD789474CEFC0165831782168610860B
:10071000178682E08187808B13861286128A118A5F
:1007200084EA9CE293838283148216820895AC014A
:10073000529542954F7045275F704527292F3327E3
:1007400024273527AC01452F552742954F70242784
:100750003527AC014F7055278FE028272F7033279E
:1007600081E04217530709F080E008958091AE00C0
:10077000813051F028F08230C1F01092AE003AC0C2
:1007800081E08093AE0036C08091B000893050F097
:1007900082E08093AE001092AD001092B2001092F1
:1007A000B10028C01092AE0025C08091B000982FF3
:1007B00093509730E8F4863038F0E1EBF0E0808138
:1007C0009181816091838083EDEAF0E080818F5F89
:1007D0008083803121F483E08093AE000BC0E1EB95
:1007E000F0E080819181880F991F9183808302C0FE
:1007F0001092AE001092B0000895CF93DF93FB01EA
:10080000EC01A881B98181E08483ED01C07FDD27FF
:10081000D695C795D695C795D695C795C258DF4F3B
:100820008881808799819187C82FD0E0C359DF4F95
:1008300088818783AA27BF70AB2FBB27AA0FBB1F56
:10084000A258BF4F8C91878711969C91908BA82FAF
:10085000B0E0A359BF4F8C918687DF91CF91089567
:10086000CF93DF93FB01EC01A881B981A07FBB2767
:10087000B295A295AF70AB27BF70AB2781E08483A0
:10088000ED01C370DD27CC0FDD1FCA58DF4F888113
:10089000808799819187C82FD0E0C359DF4F888125
:1008A0008783A695A695A370B0E0AA0FBB1FAA5890
:1008B000BF4F8C91878711969C91908BA82FB0E0A9
:1008C000A359BF4F8C918687DF91CF910895FC018A
:1008D0008181881F8827881FFB019681981719F04E
:1008E000868381E0089580E00895EF92FF920F9350
:1008F0001F93CF93DF938C01EB01DC018D919C91D1
:1009000090FF05C07B01BEE0EB0EF11C04C07B0133
:10091000E7E0EE0EF11CBE01C801D9DFD8012D9130
:100920003C91A901407F5527529542954F7045272C
:100930005F70452731FF22C11C825527FA01EF5E07
:10094000FF4F0994882309F42EC1F7018281811198
:1009500007C0118280916D00808383E0828323C170
:1009600088E0F701818380917500808312821BC12A
:10097000882309F418C1D70112969C91992319F084
:10098000913049F404C081E0F701828307C0D701A8
:1009900012961C9203C0882309F405C1F7018081D7
:1009A0008F3F09F400C18F5F8083FDC0882309F465
:1009B000FAC0D7018C91882309F4F5C081508C933B
:1009C000F2C0882309F4EFC0F7018281823020F061
:1009D0001282118280E003C08181883030F4F701F7
:1009E0009281911102C08F5F8183D70111968C9102
:1009F0001197882349F012969C911297913051F4E7
:100A0000815011968C9306C0F7018281813011F4D8
:100A100081831282D7011196EC911197F0E0E3598E
:100A2000FF4F80818C93BFC0882309F4BCC0F701BD
:100A30008281823028F081E08283118280E003C0CD
:100A40008181883030F4F7019281913011F48F5F09
:100A50008183D70111968C911197882349F01296C2
:100A60009C91129791110BC0815011968C9307C0E5
:100A7000F7018281811103C081E081838283D701E4
:100A80001196EC911197F0E0E359FF4F80818C9320
:100A90008AC088E0F701818380917500808312828B
:100AA00082C088E0D70111968C93119780917500D0
:100AB0008C9381E012968C9376C0882309F473C0DE
:100AC00088E0F701818380917500808382818111A4
:100AD00003C081E0828367C0128265C085E0F701B0
:100AE000828381E085835FC085E0D70112968C9375
:100AF000129715961C9257C0882309F454C0F70129
:100B00008581882311F0158202C081E0858385E00C
:100B1000F701828381E0868346C085E0D701129683
:100B20008C93129716961C923EC08823E1F1F70130
:100B30008681882311F0168202C081E0868385E0D9
:100B4000F70182830FC0882371F1D70112968C912F
:100B5000813041F4F701118280916D00808383E040
:100B6000828321C088E0D70111968C9311978091E0
:100B700075008C9381E012968C9315C0FA01EE0FEC
:100B8000FF1FE258FF4F8081D70111968C93119778
:100B9000918112969C931297E82FF0E0E359FF4F52
:100BA00080818C931C82DF91CF911F910F91FF90D8
:100BB000EF9008950F931F93CF93DF93EB01FC0108
:100BC0000081118184DE882309F460C0007F112731
:100BD000C801929582958F7089279F7089278230EE
:100BE000910551F134F4009779F0019709F04BC069
:100BF00013C086309105F1F18730910509F446C0A4
:100C0000049709F040C024C01C82188680916D00B2
:100C10008F8384E089873AC01C82E885E830B0F58C
:100C2000EF5FE887F0E0E359FF4F80818F8389858C
:100C3000823060F119862AC01C82E885EE2331F1EA
:100C4000E150E887F0E0E359FF4F80818F831EC0B9
:100C50001C828F85811107C088E08F878091750085
:100C60008E87188A13C01F8680916D008E8782E060
:100C7000888B0CC06D8162FF02C0637001C064602C
:100C8000CE0141DD03C06D81CE013DDDDF91CF910D
:100C90001F910F910895FC012081318136FF02C020
:100CA000ACDD089522273770311102C083DF08952B
:100CB000313011F4D5DD089532FD17DE08959C0121
:100CC00022273073232F22952F7093FD02C0822F8D
:100CD0000895822F84600895E199FECF1FBA8EBBDC
:100CE000E09A99278DB30895262FE199FECF1CBA7B
:100CF0001FBA8EBB2DBB0FB6F894E29AE19A0FBED5
:080D000001960895F894FFCF5D
:100D0800FF4F70656E50462D56312E3200001F3E43
:100D18005D7C9BBAD9FF00020800080100040002AC
:100D2800010002000300040005000600070000049B
:0E0D380007010601050104010301020101018A
:00000001FF
